:020000020000FC
:0200000071C0CD
:02000800189549
:0200160002C026
:10001A0012C00F931F930FB716B31C7041F41091BF
:10002A006000103009F003C011E0109360000FBFA8
:10003A001F910F9118950F931F932F933F934F93EF
:10004A005F935FB74091670045300CF403C04427C3
:10005A0040936700403081F4939A949A959A0EF0EF
:10006A0002C00BE002C000916500002311F09298D3
:10007A0001C0929A6ED31AD2413081F4929A949A1C
:10008A00959A0091640030916500032B11F09398C2
:10009A0001C0939A009164005CD308D2423041F4C3
:1000AA00929A939A959A94980091630052D3FED1AA
:1000BA00433041F4929A939A949A959800916600E3
:1000CA0048D3F4D14395409367005FBF5F914F9146
:1000DA003F912F911F910F9118950FED0DBF0FE7CB
:1000EA0001BB01EE07BB0CE108BB0CE302BB02E05B
:1000FA0000BF05E003BF03E206BF00E20BBF0CE14D
:10010A0000BD03E309B900E002B908E00AB906E054
:10011A0003B911241092670000E00093600004E024
:10012A00302E00D1042D003111F0B2D014C000E0FD
:10013A00302EF8D040926B0001E0302EF3D040927E
:10014A006C0002E0302EEED040926D0003E0302EBB
:10015A00E9D040926E00002700936800009369007E
:10016A0000EF00936A000FEF0093710066243ED1FE
:10017A0000916F00083209F405C012E01093600084
:10018A000FD301C006D380E090E0009160000030F8
:10019A0051F420916A002093660019D1C0D2CAD0C6
:1001AA0011E019BF41D0013009F4BCD1023069F71E
:1001BA001BE0109363001093640010936500109382
:1001CA00660011E019BFE1CFEE24FF1841E1001FDC
:1001DA00111F4A9509F40895EE1CFF1CE21AF30A4E
:1001EA0020F4E20EF31E8894F2CF0894F0CFFF18A1
:1001FA0029E0001F2A9509F40895FF1CF11A18F442
:10020A00F10E8894F6CF0894F4CF5527442760E17D
:10021A003695279510F4400F511F579547953795F6
:10022A0027956A95B9F708950F931F93009168006F
:10023A00502E2AD000916A00502E26D000B30170A9
:10024A00502E22D000916D00502E1ED000916B00CE
:10025A00502E1AD000916C00502E16D000916E00CC
:10026A00502E12D000916000502E0ED05FB60CD0E6
:10027A0004E0502E09D00027502E16E005D01A951A
:10028A00E9F71F910F9108955D9BFECF5CB8089521
:10029A0001E000936B00402E00E0302E36D00CE2D5
:1002AA0000936C00402E01E0302E2FD005E0009321
:1002BA006D00402E02E0302E28D001E000936E003F
:1002CA00402E03E0302E21D000E1402E04E0302EF3
:1002DA001CD008950F9300916B00402E00E0302E41
:1002EA0014D000916C00402E01E0302E0ED0009107
:1002FA006D00402E02E0302E08D000916E00402E94
:10030A0003E0302E02D00F910895F8940F93E199EB
:10031A00FECF00E00CBB3EBA4DBAE29AE19A0F91C9
:10032A0078940895F894E199FECF3EBAE09A4DB2D6
:10033A00789408950F931F932F933F934F935F934E
:10034A007F9300916800109169002AE030E05DDF38
:10035A00022F132F20916A003327020F131F409197
:10036A006C0050916B0060916D004F935F937727FB
:10037A00461B570BB42EA52E5F914F917727460F38
:10038A00571FD42EC52E0EF004C0009510950F5F8E
:10039A001F4FB016A10624F40D151C054CF40FC00E
:1003AA0040916E00442311F4909801C0909A07C0BE
:1003BA0040916E00442311F4909A01C090987F9165
:1003CA005F914F913F912F911F910F9108951F9324
:1003DA0061D052E135E54DEBFED112D010916800A3
:1003EA00812F10916900912F1F9108950F9349D180
:1003FA0003E3802E5BD1AFE6B0E077D10F91089589
:10040A000F931F932F933F934F933BD170FF3CC0A1
:10041A000CEC802E4BD10EEB802E48D1A8E6B0E032
:10042A0064D1A9E6B0E061D1109168002091690019
:10043A002F93287F283F11F0E89407C02F916894E2
:10044A00109520951F5F2F4F01C02F912695179564
:10045A002695179526951795269517953091680034
:10046A000EF43195432F3F70432F330F330F330F61
:10047A00440F340F369536953695369510936800A5
:10048A002093690030936A004F913F912F911F91F9
:10049A000F9108950F93F5D070FF06C00CEC802ED3
:1004AA0005D104E4802E02D10F9108950F930F9283
:1004BA000FB800E40EB90BE10DB9769BFDCFC09AD7
:1004CA00C0980F900F9108950F93B49B01C01CC060
:1004DA0000917100002309F417C0002700937100EE
:1004EA0066D16394162D143014F453D10DC010E064
:1004FA0019BF929A939A949A959A6624EBDE50D1F0
:10050A00969810E010936000B49901C009C0009158
:10051A007100002309F004C00FEF0093710047D166
:10052A000F9108950F931F932F933F934F93062D87
:10053A00002309F004C09098969A2BD16394C4DFE3
:10054A00013029F0023051F1033039F194C0E7D07B
:10055A00B29B04C000C0B39B0AC011C028D110913D
:10056A006D00183C09F0139510936D0008C01FD157
:10057A0010916D00113009F01A9510936D00E894EE
:10058A000F931F9300916D001AE031DE802F992797
:10059A00F09266001F910F916EC047C0C0D0B29B07
:1005AA0004C000C0B39B13C021C001D110916C00DC
:1005BA0020916B00103B34E0230731F03AE0130F2F
:1005CA003327231F10936C0020936B000FC0EFD0CA
:1005DA0010916C0020916B001C303EEF230711F044
:1005EA001A50204010936C0020936B000F931F93B6
:1005FA002F933F9300916C0010916B00212F20786C
:10060A0011F4E89405C06894009510950F5F1F4F88
:10061A002AE030E0D9DD802F912F0AE000936600AE
:10062A003F912F911F910F9126C0E894B29B04C06D
:10063A0000C0B39B06C009C0BAD011E010936E0087
:10064A0004C0B5D010E010936E001127812F912FAE
:10065A001EE01093630010936400109365002091CC
:10066A006E00222309F004C01CE01093660003C048
:10067A001DE0109366004F913F912F911F910F91AA
:10068A000895F894B99A33E04EEBA1D0B99830E0C6
:10069A004AE89DD005D033E042E399D07894089592
:1006AA00B19B716002C0B1997E7F0895F8940F934F
:1006BA001F93082D18E0069508F448F0B99A30E01F
:1006CA0046E785D0B99830E042E181D008C0B99AAE
:1006DA0030E04AE07CD0B99830E04EE778D01A95FD
:1006EA0051F71F910F9178940895F8940F931F93DF
:1006FA00002718E00695B99A30E04AE068D0B99820
:10070A0030E040E164D0B199006830E04CE65FD057
:10071A001A9581F70C931F910F91789408950F936E
:10072A005F9353E0A3E6B0E0809361009093620088
:10073A0000916100109162002AE030E045DDED92FF
:10074A0000936100109362005A9591F75F910F919F
:10075A0008950F931F93EAEEF7E01127E00FF11FB8
:10076A00049000916700023009F010C0002D0F7745
:10077A00002E062D02302CF400916000023029F080
:10078A0005C0002D0068002E01C0FBCF1F910F91FC
:10079A000895C59A53E039EA4DE71DD0C5980895E2
:1007AA00C59A5CE034E34DEF16D0C59808950F93CF
:1007BA001F932F932AE01FEF0FEF0A95F1F71A956F
:1007CA00D9F72A95C1F72F911F910F91089541509A
:1007DA003040E8F70895415030405040E0F708951E
:0E07EA00C0F9A4B0999282F880909CBFC68995
:00000001FF
